:020000040800F2
:10000000383100204D200008692000086D200008CC
:100010007120000875200008792000080000000009
:100020000000000000000000000000007D2000082B
:10003000812000080000000085200008031200084D
:10004000892000088D2000089120000895200008D4
:10005000992000089D200008A1200008A520000884
:10006000A9200008AD200008B1200008B520000834
:10007000B9200008BD200008C1200008C5200008E4
:10008000C9200008CD200008D1200008D520000894
:10009000BD0D0008070E0008D9200008DD2000086B
:1000A000E1200008E5200008E9200008ED20000814
:1000B000F1200008F5200008F9200008FD200008C4
:1000C0000121000805210008092100080D21000870
:1000D0001121000815210008192100081D21000820
:1000E0002121000825210008292100082D210008D0
:1000F00031210008352100083921000800000000E6
:100100003D210008000000004121000845210008B1
:10011000492100084D2100085121000855210008FF
:10012000592100085D2100086121000865210008AF
:10013000692100086D21000871210008752100085F
:10014000792100087D21000881210008852100080F
:1001500010B5DFF81416884208D140F21944200087
:1001600000F02BFB200000F03BFB07E040F21A44BC
:10017000200000F022FB200000F032FB10BD00291F
:1001800000D1FEE7C0B2002805D002282ED01AD335
:10019000032842D05AE0002048710020C871002096
:1001A000887140F2FF3048810020087200204870BA
:1001B000022088700020C87000200871002048725A
:1001C0000020087070470120C881002008740020BA
:1001D00008810020088000204880002088800020BE
:1001E000C8800020888100204881EBE7002005E0DE
:1001F00000220300DBB20B44DA72401C0200D2B2D0
:10020000082AF5D300208872002048600020087278
:100210000020487200200860D4E7002005E000229A
:100220000300DBB20B44DA72401C0200D2B2082A8F
:10023000F5D300208872002048600020087200205A
:10024000C8740020487200200860BBE7FEE730B4A5
:1002500002000B004FF6FF7001000024156835F016
:1002600002051560156855F00105156000E0491E8E
:10027000151D2D68ED0701D40029F8D1111D09685D
:10028000C90701D400246FE019785D782D0615F0B8
:10029000407555EA81759978090411F470210D4370
:1002A000D978090511F4E0010D435989491E8905E2
:1002B000890D0D4312F11C010D601979012904D13A
:1002C000116851F08001116003E0116831F0800184
:1002D00011605979012904D1116851F04001116070
:1002E00003E0116831F0400111609979012904D1CE
:1002F000116851F02001116003E0116831F0200114
:100300001160D979012904D1116831F0100111600F
:1003100003E0116851F010011160197A012904D12C
:10032000116831F00801116003E0116851F0080113
:100330001160597A012904D1116851F0040111604A
:1003400003E0116831F004011160116849084900A7
:10035000116000E0401E111D0968C90701D5002881
:10036000F8D1002800D001242000C0B230BC704772
:1003700070B400210121428911FA02F2DFF8EC3356
:10038000196851F001011960DFF8E44321689143D5
:100390002160C189002918D1DFF8D8130D68954371
:1003A0000D60C188458855EA01454189DFF8C86379
:1003B00016EBC10635608188058855EA01454189FB
:1003C000DFF8B86316EBC1063560C189012918D181
:1003D000DFF8A0130D6815430D600188458855EAC4
:1003E00001454189DFF8906316EBC10635608188CD
:1003F000C58855EA01454189DFF8806316EBC106DF
:1004000035608189002905D1DFF874130D689543A3
:100410000D6004E0DFF868130D6815430D60018975
:10042000002905D1DFF85C130D6895430D6004E0E9
:10043000DFF850130D6815430D60007C012802D1D0
:10044000206802432260186840084000186070BCB1
:10045000704730B4002210F108021268520101D531
:1004600000220EE010F108021268120101D50122EB
:1004700007E010F108021268D20001D5022200E064
:1004800003221300DBB2032B01D103208FE0130002
:10049000DBB210EB031313F5C0731B6813F00103F9
:1004A0001400E4B210EB041414F5C07423600B7A4A
:1004B000002B13D11300DBB210EB031313F5C07341
:1004C0001B680C684D7A55EA44552B431400E4B27E
:1004D00010EB041414F5C074236014E01300DBB2B5
:1004E00010EB031313F5C0731C684B680D7A55EAC3
:1004F000C3054B7A1D432C431300DBB210EB0313EF
:1005000013F5C0731C601300DBB210EB031313F57B
:10051000C2731B681B091B011400E4B210EB041426
:1005200014F5C27423601300DBB210EB031313F550
:10053000C2731C688B7A1C431300DBB210EB0313ED
:1005400013F5C2731C608B7B4C7B240454EA036458
:100550000B7B54EA0324CB7A1C431300DBB210EB71
:10056000031313F5C4731C608B7C4C7C240454EA85
:1005700003640B7C54EA0324C97B0C431100C9B209
:1005800010EB011111F5C6710C601100C9B210EB2E
:10059000011111F5C071096851F001011300DBB2BE
:1005A00010EB031010F5C07001601000C0B230BC39
:1005B000704700220022C9B2002903D002290DD0C1
:1005C00006D311E008300168DFF8BC0101400CE0FF
:1005D00008300168DFF8B401014006E00830016826
:1005E000DFF8AC01014000E0002100290CD0DFF869
:1005F000980181420AD0DFF89401814208D0DFF8E7
:100600009001814206D007E0022006E0012004E0CC
:10061000012002E0012000E00020C0B270470B0082
:10062000DBB210EB031313F5D8731B6813F004034C
:100630001372137A002B09D10B00DBB210EB0313FA
:1006400013F5D8731B685B0D136008E00B00DBB279
:1006500010EB031313F5D8731B68DB0853600B0012
:10066000DBB210EB031313F5D8731B6813F002030E
:1006700053720B00DBB210EB031313F5DA731B6834
:100680001B0AD3740B00DBB210EB031313F5DA7300
:100690001B6813F00F0393720B00DBB210EB031314
:1006A00013F5DC731B68D3720B00DBB210EB031382
:1006B00013F5DC731B681B0A13730B00DBB210EB22
:1006C000031313F5DC731B681B0C53730B00DBB2B5
:1006D00010EB031313F5DC731B681B0E93730B00F5
:1006E000DBB210EB031313F5DE731B68D3730B003F
:1006F000DBB210EB031313F5DE731B681B0A1374D4
:100700000B00DBB210EB031313F5DE731B681B0C3D
:1007100053740B00DBB210EB031313F5DE731B688D
:100720001B0E9374C9B2002907D110F10C0109689E
:1007300051F020010C30016006E010F11001096851
:1007400051F0200110300160704710F1140212685E
:10075000114314300160704710F11402126832EA3C
:1007600001011430016070470064004000660040E1
:100770001C6600400C660040406600404466004035
:1007800004660040146600400300000400030008F3
:100790000000031010B4DFF87020010009B212EB62
:1007A00091110B68012410F01F018C40234300B20B
:1007B00012EB9012136010BC704710B4DFF84820A1
:1007C000010009B212EB91110B68012410F01F0116
:1007D0008C40234300B212EB9012136010BC7047A0
:1007E00010B4DFF82420010009B212EB91110B685C
:1007F000012410F01F018C40A34300B212EB9012B1
:10080000136010BC70470000001002402DE9F8434F
:10081000040020890B28C0F21C810021200000F078
:1008200013FA05000121200000F00EFAEDB2552D5B
:1008300040F00B81C0B2AA2840F0078102212000BD
:1008400000F002FA07000321200000F0FDF9050086
:100850000421200000F0F8F90600F6B23602052166
:10086000200000F0F1F956FA80F6FFB2162F04D0FE
:100870000121200000F0FDF9EBE020892900C9B238
:1008800009318842C0F2E580DFF894735520387052
:10089000AA2078700720B8705120F8702900C9B2DA
:1008A000083189B2200000F0CFF9C0B2F0280DD095
:1008B0000121200000F0DDF90120DA490870DA4852
:1008C0004CF202318180F0218170C2E02900C9B26E
:1008D000091D89B2200000F0B7F980462900C9B28D
:1008E000491D89B2200000F0AFF981462900C9B244
:1008F000891D89B2200000F0A7F95FFA88F85FFA35
:1009000089F95FEA094919EB0869C0B219EB0029B6
:100910002900C9B2C91D89B2200000F095F959FA21
:1009200080F85FF002090AE0494689B2200000F031
:100930008BF9494689B23944887019F10109484652
:1009400080B22900C9B2091D8842EDDB2900C9B275
:10095000891D380000F0C3F9804510D00120B1494D
:100960000870B1484CF202318180F1218170EDB202
:100970000935290089B2200000F07BF969E0EDB269
:100980000935290089B2200000F073F9A54D002037
:100990006880B6B242F20550361A4BD047F6064090
:1009A000361A06D040F27A20361A23D07C3E38D050
:1009B00046E09D48817801291BD0012181700121E9
:1009C00029704CF202418180D7F80F10C16097481E
:1009D00000F052FA002005E00021954A03009BB286
:1009E000D154401C010089B2B1F5006FF4DB002046
:1009F000A8802EE08C480221817017F10D018160E2
:100A0000B97A09027A7A8918C180C188B1F5006F74
:100A100001DB0021C1804CF20221818001210170A3
:100A200017E0814803218170012129704CF20251A5
:100A300081800EE005207C4988700120287008E044
:100A40000121200000F015F903E00121200000F051
:100A500010F9BDE8F18370B5764D1121280000F042
:100A60003EF90100090E69740100090CA974010026
:100A7000090AE9742875704C70480088216808607C
:100A8000002021684872002021680872082021682F
:100A9000887228782168C8726878216808730622ED
:100AA000291D206810F10D06300000F035FA20688D
:100AB00000F038F9002821D0082021688872082227
:100AC00015F10A01206810F10B06300000F024FA3D
:100AD000206800F027F9002810D0042021688872CF
:100AE000042215F11201206810F10B05280000F016
:100AF00013FA206800F016F90028FFD070BD70B519
:100B00004F4C0B21200000F0EAF80100090EE172C1
:100B10000100090C21730100090A6173A073464D9D
:100B2000464800882968086000202968487200202B
:100B30002968087208202968887220782968C87294
:100B40006078296808730622211D286810F10D06B7
:100B5000300000F0E1F9286800F0E4F8002811D036
:100B60000620296888722868827A14F10A012868A8
:100B700010F10B04200000F0CFF9286800F0D2F843
:100B80000028FFD070BD70B52E4C020092B2120A40
:100B9000A271E071217289B2090A61720A212000F2
:100BA00000F09DF80100090EA1720100090CE1722C
:100BB0000100090A217360731F4D204800882968CD
:100BC00008600020296848720020296808720820FF
:100BD0002968887220782968C87260782968087343
:100BE0000622211D286810F10D06300000F094F94E
:100BF000286800F097F8002811D00520296888722D
:100C00002868827A14F10A01286810F10B04200088
:100C100000F082F9286800F085F80028FFD070BD48
:100C20005410002024110020101100200030000872
:100C300054080020000000204C0000203800002054
:100C400018000020280000200A00038989B28B4286
:100C500009D3C1888A181100438889B2994203D305
:100C60004188521A00E00022C06892B2805CC0B293
:100C7000704770B504000D002089290089B28842B0
:100C800016D3734E02213000FFF766FD2089401B0A
:100C9000208102213000FFF758FDE0884519280027
:100CA000618880B2884201D360882D1AE58015E002
:100CB000674E02213000FFF74FFD2589002020817B
:100CC00002213000FFF741FDE088451928006188C6
:100CD00080B2884201D360882D1AE58070BD70B45F
:100CE00000225FF0FF3200250DE05A4B1600360E51
:100CF000F6B253F8263012025A40641C23009BB20D
:100D0000042BF2DB6D1C2B000C009BB2A4B2A3429F
:100D100005D22B009BB2C35C5A400024EEE71000C2
:100D200070BC704770B5010000244B4D484E300038
:100D3000FFF78FFB287000E0641C29783000FFF774
:100D400038FC012803D04FF6FF708442F4D3297891
:100D50003000FFF72EFC4FF6FF70844203D300F003
:100D6000E3F9002000E0012070BD30B400221DE056
:100D70003A4B1B681400E4B22344DB7AC4688588CC
:100D8000635583885B1C838083884488A34201D396
:100D90000023838003895B1C038143880489A34269
:100DA00003D24388038101238372521C13000C0079
:100DB000DBB2E4B2A342DBD330BC704738B5244C7D
:100DC000264D2A6800212000FFF729FC2868007AB8
:100DD000002803D12868807A002804D1042120004B
:100DE000FFF7B3FC0EE02868006840F251718842BA
:100DF00004D12868817A1A48FFF7B7FF0421200040
:100E0000FFF7A3FC31BD38B5114C144D2A68002101
:100E10002000FFF704FC2868007A002803D1286826
:100E2000807A002804D104212000FFF78EFC0EE018
:100E30002868006840F25171884204D12868817A9C
:100E40000748FFF792FF04212000FFF77EFC31BD29
:100E500000640040EC190008341100204800002014
:100E60003800002080B500F01FFA40F2073000F093
:100E70001DFB00F03CFA01BD70B505000020002408
:100E800000F012FA00260FE009E04FF4006000FBCA
:100E9000065000F041FAC0B20328F5D1641C40F2BC
:100EA000073000F003FB761C4FF4006000FB065097
:100EB00017498842E9D300F01AFA002C01D001202A
:100EC00000E0002070BDF8B504000D001600002001
:100ED00000F0EAF9002701E0241D7F1CB74212D27E
:100EE0000C4884420FD255F82710200000F085FAF4
:100EF000002806D1206855F827108842ECD002203F
:100F000004E0032002E000F0F2F90020F2BD00004E
:100F100000E00308FCDF030862B38B0708D0521E11
:100F200011F8013B00F8013B00F024808B07F6D15B
:100F3000830740F0208000BF103A07D330B4B1E8F7
:100F40003810103AA0E83810F9D230BC530724BF4B
:100F5000B1E80810A0E8081044BF51F8043B40F87D
:100F6000043BD20724BF31F8022B20F8022B44BFE8
:100F70000B7803707047121F17D35B0009D151F82B
:100F8000043B20F8023B1B0C121F20F8023BF6D258
:100F90000BE051F8043B00F8013B1B0A20F8023B30
:100FA0001B0C121F00F8013BF3D238BF121D521E5A
:100FB00024BF11F8013B00F8013BF8D8704730B46A
:100FC000002513E050F8042BD30744BFA9F1010317
:100FD0009A18091F042942F8045BFAD213468C07B9
:100FE00044BF15809B1CC90748BF1D7050F8041BE7
:100FF0000029E7D130BC7047020052B2002A08D560
:1010000009019E4A40B210F00F00104400F8041C81
:1010100003E009019A4A40B21154704780B5411E5D
:10102000B1F1807F01D301200EE0401E9549086098
:101030000F215FF0FF30FFF7DFFF002092490860CB
:10104000072092490860002002BD80B500F011F829
:1010500000F029F801BD80B500F005F800F0D7F8E0
:1010600000F0E5F801BD80B500F0B3F800F05CF8E1
:1010700001BD80B54FF4C060FFF78CFB40F2026009
:10108000FFF788FB40F20360FFF784FB40F2046047
:10109000FFF780FB40F20760FFF77CFB40F219701E
:1010A000FFF778FB01BD10B5794C4FF48053032254
:1010B0001021200000F072FA4FF48051200000F05F
:1010C000DFFA4FF4004303224821200000F066FAC3
:1010D0004FF40041200000F0D3FA01215FF4EA1040
:1010E00000F0D1FA6B4C4FF48073032204212000EE
:1010F00000F054FA4FF4007303221821200000F08E
:101100004DFA654C022303221021200000F046FA1C
:101110000221200000F0B1FA4FF401430322102114
:10112000200000F03BFA10BD10B588B069460020E1
:10113000FFF725F803A90020FFF721F8574C2000FE
:10114000FFF706F800208DF8040001208DF8050057
:1011500000208DF8060001208DF8070000208DF892
:10116000080001208DF8090000208DF80000002003
:101170008DF8010005208DF8020000208DF8030095
:101180001220ADF80A0069462000FFF760F8002041
:10119000ADF816000020ADF818000120ADF81A00D7
:1011A0004EF62020ADF80C000020ADF80E004FF6F2
:1011B000E070ADF810000020ADF812000020ADF88E
:1011C000140001208DF81C0003A8FFF7D1F808B027
:1011D00010BD80B5324800684FF47A71B0FBF1F071
:1011E000FFF71CFF01BD2F49086008680028FCD1EB
:1011F00070472C490868002802D00868401E086023
:10120000704780B5FFF7F5FF00F072FB01BD80B5B8
:101210004FF4A06000F088FB00220321142000F0AE
:1012200088FB00220321152000F083FB01BD10B5CF
:101230001A4C02212000FFF788FA08212000FFF74E
:1012400084FA10212000FFF780FA40212000FFF7E8
:101250007CFA4FF400412000FFF777FA4FF48061E9
:101260002000FFF772FA4FF480712000FFF76DFA4B
:101270004FF400712000FFF768FA10BD18ED00E090
:1012800000E400E014E000E018E000E010E000E01E
:1012900000080140000C01400010014000640040C3
:1012A000500000202C110020DFF86C0200680006BE
:1012B00007D5DFF86802DFF868120160DFF8641212
:1012C0000160DFF86402008880B240F201218842A8
:1012D0000CD3DFF858020068000607D5DFF850028B
:1012E000DFF83C120160DFF83C1201607047DFF864
:1012F0002802016851F080010160DFF82C020088AB
:1013000080B240F20121884205D3DFF82002016853
:1013100051F080010160704770B50400DFF80802E9
:10132000008880B240F20121884247D3DFF80402EE
:1013300084421DD2DFF80052280000F009F90100B4
:10134000C9B2002957D1DFF8D061306850F00200EF
:101350003060DFF8E8010460306850F04000306031
:10136000280000F0F5F8316831F00201316042E008
:10137000DFF8C451280000F0FEF80100C9B20029CE
:1013800039D1DFF8A861306850F002003060DFF832
:10139000B0010460DFF8AC010068800702D5DFF817
:1013A0009C010460306850F040003060280000F07C
:1013B000E2F8316831F0020131601CE0DFF8785169
:1013C000280000F0C5F80100C9B2002913D1DFF8E8
:1013D0004861306850F002003060DFF8600104605E
:1013E000306850F040003060280000F0B1F83168FB
:1013F00031F002013160C0B270BDF8B504000D00DB
:101400000020DFF82401008880B240F201218842E8
:1014100033D3DFF82001844217D2DFF81C6130009B
:1014200000F096F80100C9B200293DD1DFF8E8705C
:10143000386850F0010038602560300000F088F80E
:1014400039684908490039602EE0DFF8EC60300067
:1014500000F091F80100C9B2002925D1DFF8CC7065
:10146000386850F0010038602560300000F083F8E3
:10147000396849084900396016E0DFF8BC6030007F
:1014800000F066F80100C9B200290DD1DFF88870BC
:10149000386850F0010038602560300000F058F8DE
:1014A0003968490849003960C0B2F2BD10B4194A20
:1014B00012EB90110B68012410F01F018C402343A4
:1014C00012EB9012136010BC704700201E490A688E
:1014D000D20701D5012008E00A68D20601D5032011
:1014E00003E00968490700D50220C0B27047002018
:1014F00016490A68D20701D5012008E00A68D20619
:1015000001D5032003E00968490700D50220C0B2D5
:1015100070470000002002401020024004200240DA
:1015200023016745AB89EFCDE0F7FF1F5020024054
:1015300044200240FFFF07080000FF0F1420024074
:10154000542002401C2002400C2002404C2002404B
:1015500010B504000120FFF7B8FF641E0100C9B2F6
:10156000012901D1002CF6D10100C9B2012900D115
:101570000420C0B210BD10B504000120FFF7B7FF72
:10158000641E0100C9B2012901D1002CF6D101006D
:10159000C9B2012900D10420C0B210BDF0B40024AA
:1015A000002411F00F04CD060DD5042A09D154F002
:1015B000030410F13C0212681A4310F13C052A6042
:1015C00001E022431400002523E048291FD1012215
:1015D000AA401A4010F110073A6018E01A00EA40D9
:1015E000D20715D506680F272A00D2B2920097407D
:1015F000BE432A00D2B2920014FA02F216432829FE
:10160000E3D10122AA401A4010F114073A600660A3
:101610006D1C2A0092B2082AE0D3082527E0482949
:1016200022D10122AA401A4010F110073A601BE0B3
:101630001A00EA40D20719D5021D16680F272A00A2
:10164000083AD2B292009740BE432A00083AD2B27A
:10165000920014FA02F216432829E0D10122AA408E
:101660001A4010F114073A60021D16606D1C2A0022
:1016700092B2102ADCD3F0BC704710300160704782
:1016800014300160704730B4002200220022002292
:10169000002802D51E4A146801E01E4A1468C0F3EF
:1016A000034283B210F44015B5F5401F08D1220063
:1016B00032F0E062174C256835F0E065256013E0F4
:1016C000C50207D5032515FA02F234EA020252F0E8
:1016D000E06209E00200520DD2B2120113FA02F2E6
:1016E00034EA020252F0E062C9B2002906D00100D9
:1016F000490DC9B209018B4013431A00002802D5D5
:101700000348026001E00348026030BC70470000FB
:101710001C0001400400014001B582B0029801683C
:1017200077480140B1F1005F0DD10298001D0068BB
:1017300000907448009901600299096881F3088853
:101740000068804702E00120FFF74DFD07BD80B52E
:10175000FFF788FB6C48002181700021C1800021C7
:101760000170002141700021017468484FF47A71C2
:1017700081800021418001BD80B56548FFF746F8B2
:1017800000F02EF800F043F800F012F85E484078C0
:101790000128F2D13220FFF726FD5E48FEF7D8FC83
:1017A00002215D48FFF76CFF5C48FFF7B5FFE4E7F7
:1017B00010B5554C6078002811D1A07800280ED0C3
:1017C0005248418840F6B932914208DB00214180FD
:1017D000E1884CF20230FFF7D6F90120607010BDAD
:1017E00080B549498878002810D1087C04280BDA94
:1017F00046488288322A09DB00228280087C401C0D
:101800000874FFF728F901E00120487001BDF8B520
:101810003E4C2078012826D1002020703A4DA8782F
:10182000012806D0022809D003280CD0052811D0A1
:1018300019E00021A888FFF7A6F914E0E988A88834
:10184000FFF7A1F90FE00021A888FFF79CF901201C
:10185000687008E0FFF753F90020A8700020687056
:1018600000202874FFE7284D287801283FD1002068
:101870002870E88840F60101884233DAE8880028B9
:1018800030D0274EE888304410F8010C00281ED1D3
:101890002022A968E8888027224B07FB0030FFF749
:1018A00012FB002809D0EE214CF20260FFF76BF921
:1018B0004FF47A70FFF797FCF5E70120E98831448F
:1018C00001F8010C01202070002060800FE0E98801
:1018D0004CF20220FFF757F9E1214CF20260FFF7CA
:1018E00052F904E0E2214CF20260FFF74CF9F1BD3D
:1018F00006488188491C81804188491C4180704785
:101900000000FE2F301100201011002024110020B3
:101910003800002000640040001001400030000842
:1019200054080020802F00082C4908432C490860E7
:10193000704770B504000D00160000200020002044
:101940002748016811F4E061B1F5E06F02D1002091
:10195000042129E0016811F4E061B1F5C06F02D102
:101960000120032120E0016811F4E061B1F5A06FCE
:1019700002D10220022117E0016811F4E061B1F503
:10198000806F02D1032001210EE0006810F4E060B6
:10199000B0F5407F02D10420002105E04FF4A060A3
:1019A000FFF7C2FF02200221EDB2D0F10400854012
:1019B000F6B20F20D1F10401C840064035432D0195
:1019C00008482100C9B24554012114F01F0081408C
:1019D0000548E4B2641140F8241070BD0000FA0517
:1019E0000CED00E000E400E000E100E00000000099
:1019F000B71DC1046E3B8209D926430DDC76041362
:101A00006B6BC517B24D861A0550471EB8ED0826F8
:101A10000FF0C922D6D68A2F61CB4B2B649B0C3595
:101A2000D386CD310AA08E3CBDBD4F3870DB114C42
:101A3000C7C6D0481EE09345A9FD5241ACAD155F25
:101A40001BB0D45BC2969756758B5652C836196A2E
:101A50007F2BD86EA60D9B6311105A6714401D7919
:101A6000A35DDC7D7A7B9F70CD665E74E0B62398C3
:101A700057ABE29C8E8DA191399060953CC0278B2D
:101A80008BDDE68F52FBA582E5E66486585B2BBEB4
:101A9000EF46EABA3660A9B7817D68B3842D2FADD1
:101AA0003330EEA9EA16ADA45D0B6CA0906D32D474
:101AB0002770F3D0FE56B0DD494B71D94C1B36C7A9
:101AC000FB06F7C32220B4CE953D75CA28803AF2B2
:101AD0009F9DFBF646BBB8FBF1A679FFF4F63EE10D
:101AE00043EBFFE59ACDBCE82DD07DEC77708634D2
:101AF000C06D4730194B043DAE56C539AB06822741
:101B00001C1B4323C53D002E7220C12ACF9D8E127F
:101B100078804F16A1A60C1B16BBCD1F13EB8A01B4
:101B2000A4F64B057DD00808CACDC90C07AB977841
:101B3000B0B6567C69901571DE8DD475DBDD936B84
:101B40006CC0526FB5E6116202FBD066BF469F5E65
:101B5000085B5E5AD17D1D576660DC5363309B4D38
:101B6000D42D5A490D0B1944BA16D84097C6A5ACC6
:101B700020DB64A8F9FD27A54EE0E6A14BB0A1BF8C
:101B8000FCAD60BB258B23B69296E2B22F2BAD8ABB
:101B900098366C8E41102F83F60DEE87F35DA99970
:101BA0004440689D9D662B902A7BEA94E71DB4E033
:101BB000500075E4892636E93E3BF7ED3B6BB0F308
:101BC0008C7671F7555032FAE24DF3FE5FF0BCC6E9
:101BD000E8ED7DC231CB3ECF86D6FFCB8386B8D52C
:101BE000349B79D1EDBD3ADC5AA0FBD8EEE00C690C
:101BF00059FDCD6D80DB8E6037C64F643296087A12
:101C0000858BC97E5CAD8A73EBB04B77560D044F64
:101C1000E110C54B383686468F2B47428A7B005CE5
:101C20003D66C158E4408255535D43519E3B1D259E
:101C30002926DC21F0009F2C471D5E28424D1936D5
:101C4000F550D8322C769B3F9B6B5A3B26D615031A
:101C500091CBD40748ED970AFFF0560EFAA0111069
:101C60004DBDD014949B93192386521D0E562FF10F
:101C7000B94BEEF5606DADF8D7706CFCD2202BE25D
:101C8000653DEAE6BC1BA9EB0B0668EFB6BB27D7A0
:101C900001A6E6D3D880A5DE6F9D64DA6ACD23C4A1
:101CA000DDD0E2C004F6A1CDB3EB60C97E8D3EBDB0
:101CB000C990FFB910B6BCB4A7AB7DB0A2FB3AAED9
:101CC00015E6FBAACCC0B8A77BDD79A3C660369B1E
:101CD000717DF79FA85BB4921F4675961A163288DD
:101CE000AD0BF38C742DB081C330718599908A5DF2
:101CF0002E8D4B59F7AB085440B6C95045E68E4E71
:101D0000F2FB4F4A2BDD0C479CC0CD43217D827BEB
:101D10009660437F4F460072F85BC176FD0B866884
:101D20004A16476C93300461242DC565E94B9B111D
:101D30005E565A1587701918306DD81C353D9F02B4
:101D400082205E065B061D0BEC1BDC0F51A6933751
:101D5000E6BB52333F9D113E8880D03A8DD0972408
:101D60003ACD5620E3EB152D54F6D4297926A9C592
:101D7000CE3B68C1171D2BCCA000EAC8A550ADD63C
:101D8000124D6CD2CB6B2FDF7C76EEDBC1CBA1E3A7
:101D900076D660E7AFF023EA18EDE2EE1DBDA5F0C0
:101DA000AAA064F4738627F9C49BE6FD09FDB889EF
:101DB000BEE0798D67C63A80D0DBFB84D58BBC9AB8
:101DC00062967D9EBBB03E930CADFF97B110B0AF55
:101DD000060D71ABDF2B32A66836F3A26D66B4BC7C
:101DE000DA7B75B8035D36B5B440F7B180B54B48C2
:101DF000016851F4700101604949086850F0010020
:101E0000086008688007FCD5464A106850F08000DA
:101E100010600020009002E00098401C00900098A4
:101E20005028F9D3106850F0900010600020009006
:101E300002E00098401C009000985028F9D31068E8
:101E40008008800010600B68374803400B605FF427
:101E50007F00364B1860086830F48020086000204E
:101E6000106000203249086000F001F801BD80B523
:101E700000F001F801BD10B40022002028490868D4
:101E800050F001000860521C086810F002000028A1
:101E900002D1B2F5A06FF6D10868800700D4FEE742
:101EA0002448026852F080520260234A106850F4BD
:101EB000404010601B4B186818601868186018685C
:101EC00050F4806018601C681C4804401C601C684A
:101ED0001B4804431C60086850F080700860086864
:101EE0008001FCD5106850F48030106015480168FE
:101EF000C903FBD5116851F40031116001688903F1
:101F0000FCD51868800880001860186850F002003E
:101F1000186018680007FCD510BC704788ED00E019
:101F20000010024004100240FFFFF6EA08100240D1
:101F30002C1002401C10024000700040FFFFC39FA5
:101F4000000004200470004030B501688468421825
:101F5000416802EB5103C90703D54C4401E0491C19
:101F600005D19A420AD012F9011B12F8015B00292F
:101F700004F8015BF3D4491EF7D5F2E70C3030BD0D
:101F800010B5074979441831064C7C44163404E0F6
:101F90000A68081D114488470146A142F8D110BDC6
:101FA0002C000000480000004EF68851CEF20001DF
:101FB000086840F470000860BFF34F8FBFF36F8F65
:101FC0004FF00070E1EE100A70470000F3EFFFFFE2
:101FD000E410000054000020000000006DFFFFFF2F
:101FE000A8010000920000000000002000F00DF8A1
:101FF000002801D0FFF7C4FFAFF300800020AFF34B
:10200000008000F004F800F00EF80120704780B561
:1020100072B6FFF71AF8FFF71EF862B6FFF797FBE4
:10202000FFF7AAFBFEE700F001B8000007463846BC
:1020300000F002F8FBE7000080B5AFF30080024A31
:1020400011001820ABBEFBE72600020001488047C4
:1020500001480047ED1D00085D200008AFF3008037
:10206000FFF7A2FFFFF7C2FFFFF7FEBFFFF7FEBFBC
:10207000FFF7FEBFFFF7FEBFFFF7FEBFFFF7FEBF94
:10208000FFF7FEBFFFF7FEBFFFF7FEBFFFF7FEBF84
:10209000FFF7FEBFFFF7FEBFFFF7FEBFFFF7FEBF74
:1020A000FFF7FEBFFFF7FEBFFFF7FEBFFFF7FEBF64
:1020B000FFF7FEBFFFF7FEBFFFF7FEBFFFF7FEBF54
:1020C000FFF7FEBFFFF7FEBFFFF7FEBFFFF7FEBF44
:1020D000FFF7FEBFFFF7FEBFFFF7FEBFFFF7FEBF34
:1020E000FFF7FEBFFFF7FEBFFFF7FEBFFFF7FEBF24
:1020F000FFF7FEBFFFF7FEBFFFF7FEBFFFF7FEBF14
:10210000FFF7FEBFFFF7FEBFFFF7FEBFFFF7FEBF03
:10211000FFF7FEBFFFF7FEBFFFF7FEBFFFF7FEBFF3
:10212000FFF7FEBFFFF7FEBFFFF7FEBFFFF7FEBFE3
:10213000FFF7FEBFFFF7FEBFFFF7FEBFFFF7FEBFD3
:10214000FFF7FEBFFFF7FEBFFFF7FEBFFFF7FEBFC3
:10215000FFF7FEBFFFF7FEBFFFF7FEBFFFF7FEBFB3
:10216000FFF7FEBFFFF7FEBFFFF7FEBFFFF7FEBFA3
:10217000FFF7FEBFFFF7FEBFFFF7FEBFFFF7FEBF93
:10218000FFF7FEBFFFF7FEBF1055AA07150C0BC1E6
:10219000094D432056312E332E30FC000DF0000047
:1021A00055AA07150C05A90341434BFC0006F05541
:1021B000AA07150C04F80005F00015070008F80040
:1021C0000F54000020E8100020FC10002000A24A5C
:0121D000040A
:040000050800205D72
:00000001FF
